:030000000219FDE5
:03000B000200AA46
:03002B0002019C33
:03005B0002034F4E
:0300730002033550
:1000800002030406080C10182030406080040608A3
:100090000C10182030406080A0C000070F1F3F0DDB
:1000A0000D04050D050305030302C2AF306308C24A
:1000B00063857C8AD2AF32C0D0C0E0206227E525BC
:1000C0006002E473E525F4C3334009758A00D26306
:1000D000F57C01D6F58A758B00758D00D262D0E073
:1000E000D0D0D2AF32C3E526334009758A00D2633F
:1000F000F57C01F6F58AC262E526F4603C306803BF
:10010000207213758B00758D00D0E0D0D0C295C2DF
:1001100094C293D2AF32C295C294C293206E0D2086
:10012000660A7414D5E0FDE57EF45290758B007577
:100130008D00D0E0D0D0D2AF32758A00D263757C0A
:1001400000C28DD262212C01C4306805206602D223
:100150009501C4306805206602D29401C430680558
:10016000206602D29301C4D29230680A20660774D6
:1001700010D5E0FDD29501C4D29130680A206607FF
:100180007410D5E0FDD29401C4D290D29230680AA6
:100190002066077410D5E0FDD29301C4C2AFC2AD92
:1001A00053E6EFC0D0C0E0D2D3D2AFE57D6009E521
:1001B0007A6005757A0041E2757A01C2CEE52A605F
:1001C00007207449152A410D7800790020742EE526
:1001D00080307E01F430E70278FF53DACF207E03CF
:1001E00043DA20307E0343DA10C2D8C271E5803092
:1001F0007E01F430E70279FFC3E89970CB306103E8
:10020000752A18207403752A18885FD27020740D1F
:10021000E52B6004152B411D43DA01C2D820700282
:10022000417BA85F206102C2702074367982B704D6
:1002300031C3E894F0400374F0F8E8C4540F28F890
:100240007984B703024162C313C3138721200802D4
:10025000C313200A06C3C898F8416228F8500374F3
:10026000FFF88822E52D54066011E533C313C3134C
:1002700024062522F52250037522FF7882B6045900
:10028000852224A824C3E52495644002A864C3E819
:1002900095664002A8668825E569700241CCC3E8EE
:1002A000AA699A5003E8FAE4F9EAC333FBE56BF470
:1002B0005B29400D256AF8E56A6002156A400B412A
:1002C000CC0AC3E56A9A5002056A78FF8826C26E96
:1002D000C3E52694F84002D26EC3E525944040025F
:1002E000D26420CF0AD0E0D0D043E610D2AD32C2E3
:1002F000CF053AE57D6009E57B6005757B00612BE4
:10030000757B017801E52A6005307402152AC3E582
:100310005F94014005756200612B756300756C0088
:10032000E5622401F56250037562FFD0E0D0D0434E
:10033000E610D2AD32C2AFC0D053E67FC260759135
:1003400000855694855795759104D0D0D2AF32C2AE
:10035000AF53E6EFC2ADC0D0C0E0C0F0D2D3D2AF51
:10036000A8FBA9FCE57D6007C3E913F9E813F8C20F
:10037000D830710261C153DACF207E0343DA1030E6
:100380007E0343DA20D271E580307E01F420E7025B
:10039000619888278928A1EE53DACF207E0343DABB
:1003A00020307E0343DA10C2D8C271307402A1DA61
:1003B0007800E580307E01F430E702A1DA885FA1A1
:1003C000C253DACF207E0343DA20307E0343DA10B3
:1003D000C271206102819A53DACF207E0343DA1082
:1003E000307E0343DA20C2D8D271885A895BC3E8D1
:1003F0009558F8E99559F97B007E087A00C3E8948E
:100400008CE994005005755E00818C882178A2E605
:10041000A8216055C3E894C8E994005008E4D2E4E8
:10042000FB7A0A8167C3E89468E994015008E4D232
:10043000E3FB7A0F8167C3E894D0E994025008E4A3
:10044000D2E2FB7A1E8167C3E894A0E994055008C4
:10045000E4D2E1FB7A3C8167C3E89498E9940850C0
:1004600008E4D2E0FB7A787E00C3E8955CFCE9956D
:0F0470005DFD30E70AECF42401FCEDF43400FDEF
:10047F00755E00C3EC9AED9E5003755E01885C8932
:10048F005D855A58855B597802A1C2C3E89527F854
:10049F00E99528F9307C02A1A6307B02A1A6307A1B
:1004AF0002A19F20750281BDE9FDE8FC81DCE9C353
:1004BF0013F9E813F8307902A19FE9C313F9E81390
:1004CF00F8307802A19FE9C313FDE813FC20612CDB
:1004DF00C3EC941CED9402400281F3ED701EC3EC4B
:1004EF0094C850180529E52970021529C3E52994E8
:1004FF000A5002A1DA755F00D270A1DAE529600215
:10050F0015297888E6F97400207F087896B90302D8
:10051F00789EE624FAFEE43400FFC3EC9EFCED9FC8
:10052F00FD9208B90310A2085007207609D276A1D0
:10053F0045307602C276A2085016B9030DECF424AA
:10054F0001FCEDF43400FD02055F78007900A1A6EF
:10055F00B90315EC33FCED33FDC3EC940AFCED94B9
:10056F0000FD50047C007D00C3EC94FFED9400402F
:10057F000678FF7900A1A6EC8575F0A4C5F0A2F767
:10058F0033F8790040030205C278FF79000205C2F3
:10059F00E9C313F9E813F8307C0EE9600278FFC362
:1005AF00E81338F8E43400F9C3E894FFE994004005
:1005BF000278FF885FD270206102A1DA741FF455B0
:1005CF002F4BF52FC274EB7002D274752A1830744A
:1005DF0003752A0A306102A1EE20740353DAFE205C
:1005EF007403752B06D0F0D0E0D0D0D2AD43E61017
:1005FF0032790102061E790302061E790A02061ECF
:10060F00791E02061E796402061E79C802061E783C
:10061F0017E4D5E0FDD8FAD9F6227A147B780206D2
:10062F00457A107B8C0206457A0D7BB40206457A1B
:10063F000B7BC80206457902B27DE4D291D5E0FD6D
:10064F00D294D5E0FDC294D5E0FDC291D5E0FDD2A4
:10065F0095E576D5E0FDC2957496D5E0FDD9D9EA3A
:10066F00F8D5E0FDD8FBDBCED29122C37C007D0014
:10067F0075F00005F0EA33FAEB33FB50F6EB13FBA2
:10068F00EA13FAC3E9FFE8FEE89AF8E99BF9500488
:10069F00EFF9EEF8B3EC33FCED33FDD5F0DFEDF908
:1006AF00ECF822E889F08A20D2D4F8A9F07B003048
:1006BF00F70B7BFFF42401F8E9F43400F9E8852007
:1006CF00F0A4ADF0F8E98520F0A4AFF0FEED2EF91F
:1006DF0074003FFA7C04C3EA13FAE913F9E813F83C
:1006EF00DCF48BF030F70AE8F42401F8E9F4340075
:1006FF00F9E889F0C2D4F8A9F0227882B60403028F
:10070F000764C3E55F9401400302072E852224E4AA
:10071F00F545F546F547F548F549C26D020764788A
:10072F0082E6FCD26DE522F523783879C7AA40AB73
:10073F0041C3EB13FBEA13FAEC146013C3EB13FB87
:10074F00EA13FAEC14146007C3EB13FBEA13FAD1A4
:10075F007A8845894622C3E5459523F8E5469400F6
:10076F00F9500CC3E89480E994FF4016020795C333
:10077F00E8947FE994005003020795787F7900028F
:10078F000795788079FF884A894B22E54A2547F8F3
:10079F00E54B3548F9854B20E4300701F43549FA2C
:1007AF0030E709C3EA94F040150207D3C3EA940F68
:1007BF0050030207D378FF79FF7A0F0207D378002F
:1007CF0079007AF0C3E5249564500AC37401952427
:1007DF00500B0207F1E54B20E70E0207F1E54B3016
:1007EF00E706884789488A492278A4E6FAC3E54A8A
:1007FF0033F8E54B33F91206B2E930E70BC3E8944F
:10080F0080E994FF4013012CC3E8947FE9940050D2
:10081F0002012C787F7900012C788079FFE820E79E
:10082F0015C3E52398F84009C3E894014003020873
:10083F00537801020853E8F424012523F8400302FA
:10084F00085378FF884C2278A5E6FAA848A94912E0
:10085F0006B2E930E70CC3E89401E994FF401602B1
:0E086F000888C3E894FFE9940050030208884B
:10087D0078FF7900020888780179FFE920E715C330
:10088D00E54C98F84009C3E8940140030208AF789D
:10089D00010208AFE8F42401254CF840030208AF2B
:1008AD0078FF88242278FFC26420693D206A12D225
:1008BD0064C3E541940A4009C3E52594405002C242
:1008CD006479A1E76023E541601F74FF8541F084E1
:1008DD008539F0306A0375F005A4F8C5F06002782B
:1008ED00FFC3E895675002A867886622C3E5409468
:1008FD00C8E5419400E566500314210A046002F531
:10090D0066220209122275E890227883E6FFE5E857
:10091D0020ECF7A8BDA9BE0573C3E573940840523A
:10092D00757300E9FA79A0E76044EA7007E5746031
:10093D001B02094DC3E895746010E5745006600CF8
:10094D00140209590460F9020959E574F574C39448
:10095D0072401B7564C0C394044013756480C394C6
:10096D0004400B756440C39404400375640075BB6B
:10097D000622E5642410500274FFF5647982B704F1
:10098D000221A6C3A864E524985002A824C3E895C3
:10099D00664002A86688258826E573B4070375BBF3
:1009AD001022743279A687F0A4C5F0A2F733F8C3EC
:1009BD00E895644002A864882288248825882688C2
:1009CD0067227540007541F022C2AF75C820A8CCD2
:1009DD00A9CDAA3A30CF010A75C824D2AFC3EA1304
:1009ED00FAE913F9E813F8AB3BAC3C883B893CC3FF
:1009FD00E89BF8E99C20690A547FF930670241F9B8
:100A0D004156AD3D8A3DF9EA9D547FFA600478FF69
:100A1D0079FFAE3EAF3F8B3E8C3FC3EC9FFCC3E9ED
:100A2D009CF542A83BA93CC3E89EF8E99FF9C3E5B4
:100A3D004113FBE54013FAE82AF540E93BF5415037
:100A4D00067540FF7541FF41A0AA40AB41AC40ADDA
:100A5D00417E047F02C3EB940440021E1FC3EB943E
:100A6D000840021E1FC3ED13FDEC13FCDEF7C3EAB5
:100A7D009CFAEB9DFBEF6009C3E913F9E813F8DF6E
:100A8D00F7EA28FAEB39FB8A408B4150067BFF8B46
:100A9D00408B41C3EB94025002D2673069047F034F
:100AAD0041CB7892E6FFC3E537948240110FC3E541
:100ABD003794A040010FC3EF940640027F057E03DB
:100ACD00E541C4540FF9E541C454F0F8E540C45470
:100ADD000F28F8C3E89EFAE99400FB4009C3EA9495
:100AED0002EB940050047A02E4FB6145AA40AB414D
:100AFD00EBC4FEEAC4540F4EFCC3EA9CFAEB94001F
:100B0D00FBC3E813C313F8EA28FAEB3400FB8A4061
:100B1D008B41C3EB94024002C2677803EBC4FE7BAA
:100B2D0000EAC4540F4EFAC3EA98FA4005C3940282
:100B3D0050027A027892E6FF306002614585525686
:100B4D00855357D26043E680C3E49AF8E49BF9C31A
:100B5D00E833F8E933F930670261E6E8FAE9FBD3E7
:100B6D00E913FDE813FC88528953C3EF94036038F1
:100B7D00EF20E00DE82CF8E93DF9ECFAEDFB020B66
:100B8D00A1E828F8E939F9C3E82402F8E93400F9B5
:100B9D007AFE7BFFC3EF9403400E8A548B55884E2B
:100BAD00894F8C508D51811A885489558A4E8B4F9F
:100BBD008C508D51306920C3E53394034019E542C3
:100BCD00A2E713F8E555F4240138400B20E708752A
:100BDD0054FFF42401F555811AE8FAD3E813FC8883
:100BED0052C3EF94036020EF20E007E82CF8ECFAF5
:100BFD008106E8282402F87AFEC3EF940340088AA0
:100C0D0054884E8C50811A88548A4E8C50E56BC393
:100C1D00335002646BF56B3060028124753404D25D
:100C2D006043E680E52D5406601FA840A941C2AF80
:100C3D0053E67F759100C3E498F594E499F59575A5
:100C4D009104D26043E680D2AF22D265754400751F
:100C5D002000306B03752040020C76D26575440080
:0D0C6D00752040306B03752000D2AF780178
:100C7A00206722E52D54066002C265C3E54194054A
:100C8A0040137802940540087803940540027806D8
:100C9A00306902780A206019E544601530690AC390
:100CAA00E53394034003D53406D2AFD26CA15891F0
:100CBA002CD2AF0000C2AF20672AE541C3FB940FD4
:100CCA0040027B0FEB240530730123306A0274283B
:100CDA0020620123F93069027982E58D13E58B13CD
:100CEA00C39940B10544E59B5440B52002A1423066
:100CFA00690A08C3E8940A400108819F20650281B5
:100D0A0076C26553E67F7591003067107594007559
:100D1A0095FC759104D26043E6808176AE40AF417E
:100D2A00C3EE33FEEF33FF50047EFF7FFFC3E49E22
:100D3A00F594E49FF595A11CC3E533940250028112
:100D4A00763065028176D802A156819FC26C53E63D
:100D5A007F759100855494855595759104854E56F5
:100D6A00854F57D26043E680D2AFE52D540660081E
:100D7A00206A020533020D92306C0D206B0A206541
:100D8A000715811581021613227800306405306533
:100D9A00027801E53775F007A4F9E5F028F5F0E9DE
:100DAA00A2F013A2F113A2F213F537C394785003F9
:100DBA00753778C3E53795384008D266C295C2942C
:100DCA00C293306002A1CC855056855157D26043F8
:100DDA00E68022207D11C2AF754302D291C292D21F
:100DEA00AF759F11020FB4C2AF754302D291C29080
:100DFA00D2AF759F11020FB4307245207D22C2AF67
:100E0A00754303900178757E02C293D290D29230D4
:100E1A006204D294C122C291D2AF759F01020FB46B
:100E2A00C2AF754303900178757E02C295D29230A3
:100E3A006204D294C142C291D2AF759F21020FB40B
:100E4A00207D17C2AF754303900153C293306202EB
:100E5A00D294D2AF759F01020FB4C2AF754303900B
:100E6A000153C295306202D294D2AF759F21020F0C
:100E7A00B4207D11C2AF754304D292C290D2AF752D
:100E8A009F21020FB4C2AF754304D290D292C2928C
:100E9A00D2AF759F01020FB4307243207D20C2AFDA
:100EAA00754305900167757E04C294D2913062043D
:100EBA00D295C1C0C292D2AF759F11020FB4C2AF10
:100ECA00754305900189757E01C294D291306204FE
:100EDA00D293C1E0C290D2AF759F11020FB4207DA8
:100EEA0017C2AF754305900149C294306202D29588
:100EFA00D2AF759F11020FB4C2AF75430590015D61
:100F0A00C2943062EBD293D2AF759F11020FB42014
:100F1A007D13C2AF754306D290D292C291D2AF75F9
:100F2A009F01020FB4C2AF754306D292C291D2AFEB
:100F3A00759F21020FB4307244207D20C2AF7543E1
:100F4A0001900189757E01C295D292306204D293D2
:100F5A00E15EC290D2AF759F21020FB4C2AF754352
:100F6A0001900167757E04C293D290D292306204D6
:100F7A00D295E180C292D2AF759F01E1B4207D166D
:100F8A00C2AF75430190015DC295306202D293D21D
:100F9A00AF759F21E1B4C2AF754301900149C29375
:100FAA00306202D295D2AF759F01C2662290014784
:100FBA00757E00C295C294C293D292D291D290C247
:100FCA006222788076090876090876040876FF088E
:100FDA0076030876FF08760A08760308760108760B
:100FEA0001788C76010876FF0876FF0876FF087686
:100FFA00FF0876FF0876030876FF0876FF0876FF73
:10100A000876250876D008762808765008760408E7
:10101A0076FF08760208760008767A0876FF087660
:10102A0001087601087600087603227887E6FFC26F
:10103A0072BF0302D2727888E6C394036008C27D45
:10104A00E630E102D27DC27E7889E630E102D27EC4
:10105A00C3EF94026008758E01D27302106D758E0B
:0F106A0000C273227880E6149000809378A4F679
:101079007881E6149000809378A5F67886E6149036
:10108900008D9378A6F6789CE67538FF75390CB40F
:1010990002067538A075390AB403067538827539A0
:1010A9000578A3E61490009A93F569120FB72222E6
:1010B9007896E6FA7897E6FB7888E6B40305C3EBF9
:1010C900940EFB307F047A007BFFC3EB9AFCC39438
:1010D9008250027C827575000575EC8575F0A4C394
:1010E900E5F0947D40F222D27F11B912060F7A0001
:1010F9007B007C10120605E55F2AFA74003BFBDCD5
:10110900F37C04C3EB13FBEA13FADCF7FEC27F118D
:10111900B922E5EF20E6037520000520903FFFE5A1
:1011290020146006901FFF1460009304600375EF9C
:101139001253D9BF7581C043FF8012060075EF02B3
:1011490043B203E5B3240420E70DF521E5E320E0EC
:10115900068521B343E301120FB77580FF75A4001B
:1011690075F19075D47F75908775A5BF75F2BF75B8
:10117900D50075A60175E241E4F8F6D8FD756B0155
:10118900120FCC12165D78988676753001C2AF12AF
:10119900061912062912060F12063012060F120638
:1011A9003712060FC2AF78FA79FA308707D9FBD818
:1011B900F7021C001135116E11B811B978988676AD
:1011C900120FB775A90075B680757D0075885075C1
:1011D900891275C82475910475D84075A82275B807
:1011E9000275E690759B80759D0075D10E75BC588A
:1011F90075BB0675BA1175E880120600D2AF1209DF
:101209000F53DACF207E0343DA20307E0343DA100E
:1012190043DA01C2D8C271120619D2617B037A0C72
:10122900E55E70077A0CDB030211AD12060F207020
:10123900030211ADC270E55FC3940240E1E52F548A
:101249001F856160F561B560D5DAD5C26153DACF22
:10125900207E0343DA20307E0343DA10C2D8C271FC
:1012690078A2E67008D274E52F54E0F52FC275759F
:101279002900120614307409C3E529940A4002D2E0
:101289007512060578023074027800C3E55F98404C
:10129900F0C2AF120629120629120629D2AF120688
:1012A90019754D007888E6B40302618B120605783A
:1012B9008CE6C39401500302138BE530C3940150AB
:1012C9000302138B207435C3E55F94FF50030213A7
:1012D9008BC2AF12063ED2AF120614C3E55F94016A
:1012E90050EFC2AF12062912060A120629D2AF120E
:1012F9000614C3E55F94FF40E90218057F02D27F17
:1013090011B9120614C2AFC27F11B9AE5FC3E55F4E
:10131900947FD2AF4076120600C2AF12063ED2AF1A
:10132900DFDC11F0C3EE94057897F6120619121650
:101339009F1217887F0AD27F11B9120614C2AFC251
:101349007F11B9AE5FC3E55F947FD2AF50E6120655
:1013590000C2AF12062912060A120629D2AFDFD639
:1013690011F0EE24057896F612061912169F121737
:10137900B712061411B9C3E55F94FF500241CD02BB
:101389001805C3E55F954D4003855F4D1206147836
:10139900017988E7B403027805C3E55F9840024103
:1013A900ADC2AF12063E12063E12063ED2AF12067B
:1013B90019753000E4F531F5320531E531F470394C
:1013C9000532789AE67819146012783214600D782B
:1013D9007D14600878FA146003753200C3E5329809
:1013E900401715327531B478998676C2AF12063E28
:1013F900D2AF7898867612061412060AE52A700585
:1014090030740221AD78012074027806C3E55F9833
:1014190040A77888E6C394036003120614E52A708E
:10142900030211ADC2AF120FB7E4F522F523F5247B
:10143900F525F526F56AD2AF7885E6C333F568E474
:10144900F545F546F547F548F549F573F52CF52DBC
:10145900F53775730875BB10120600120913E5E814
:0D14690020ECFBA8BDA9BEE97001F8887455
:1014760012091775730875BB107887E6FE76021198
:10148600357887EEF6C2AF7564FF1209AF85226420
:10149600852265852266D2AF7522017524017525E0
:1014A6000175260185636C756D0175B69075A90386
:1014B600757D017888E6B40307C27D307602D27D59
:1014C600D268D269753300120F19120F401209CF74
:1014D6001209D61209CF1209D61209CF0214F1C287
:1014E600AF1135D2AF75730075BB06120C681207C3
:1014F60009120D93120DDD1209D6120C57306D0329
:101506001207652067031208B23067031208F91242
:101516000D93120E021209D6120C68306D031207D3
:101526009A120D93120E7B1209D6120C57306D03C8
:101536001207F8120D93120EA21209D6120C683079
:101546006D03120856120D93120F191209D61209BD
:1015560013120C57120D93120F401209171209D6C7
:10156600306935206B3285676485676585636C7580
:101576006D0179187A0CC3E53399400FC269D26AB6
:101586008A3585676485676602159EC3E55F9401A3
:1015960040030214F102161B306A1B206B18E53556
:1015A600147004C26A81E5F535C3E55F9401400312
:1015B6000214F102161B753600C3E56278FA9850DC
:1015C60054307404E52A604D7888E6B40317207D0C
:1015D60005207607A1EB307602A1EB206B07D26BD4
:1015E600856764A13078F0306B058567647820C321
:1015F600E54198500281F1306B1BC26BC27D30769B
:1016060002D27DD26A75351285676481F10536E5A9
:101616005F6002C11E753600C2AF120FB77887E64B
:10162600FE760211357887EEF6E4F522F523F524E9
:10163600F525F526F568C26875A90075B680757D2D
:1016460000D2AF120600120FB7307409C3E5369404
:1016560005400221AD61BD901A0D78201216E1E514
:1016660020B4550CA31216E1E520B4AA0302167F96
:10167600120FCC12169F02169E901A0378807B0AD0
:101686001216E1A308DBF9901A0F788C7B18121654
:10169600E1A308DBF9901A2722C2AF12172012160F
:1016A600FA901A00740E1216E6A374041216E6A334
:1016B60074141216E6901A0378807B0A1216E5A3B4
:1016C60008DBF9901A0F788C7B181216E5A308DB55
:1016D600F9121733121711901A2722E493F622E60D
:1016E600438F01538FFD75EF0275B7A575B7F1F0FE
:1016F600538FFE22438F02438F0175EF0275B7A504
:1017060075B7F1901A0DF0538FFC22901A0D74558F
:10171600D1E6901A0E74AAD1E6227A3079D07820D2
:10172600901A40D1E1E520F709A3DAF7227A307959
:10173600D0901A40E7D1E609A3DAF922AB77A87868
:10174600BB01027980BB02027981BB03027982BBAD
:1017560004027984BB05027986BB06027992BB072F
:10176600027987BB080279A3BB0902799CBB0A02EE
:101776007988BB0B027989E8F7227C05120619DC09
:10178600FB22C2AF12062912063012063712063E97
:1017960012060A12062912063012063712063E12E1
:1017A600060A12062912063012063712063ED2AF74
:1017B60022C2AF12063E1206371206301206291250
:1017C600060A12063E1206371206301206291206BD
:1017D6000A12063E120637120630120629D2AF2228
:1017E600AE77AF78C2AF1206291206291206291261
:1017F600060ADEF212063E12060ADFF8D2AF2212FF
:101806001788121780121780757701757801757918
:10181600001217E67C05AD5F120619C3ED955F70E1
:10182600F5C3E55F9401400AC3E55F94FF403702C4
:10183600184912174212169F121788C2AF75EF1277
:10184600121780DCD10579C3E5799403500280C173
:101856001217800578E5771490009F93F808C3E582
:0F1866007898500280A81217801217800577C358
:10187500E577940C50028094120FCC12169FC2AFDC
:0618850075EF121217803E
:0319FD0002111BB9
:101A00000E0414090904FF03FF0A03010155AA018A
:101A1000FFFFFFFFFF03FFFFFF25D0285004FF0259
:081A2000007AFF01010003FF41
:101A4000234F76736B794D5232304150726F2320A1
:101A500023424C48454C492346333930232020202B
:101A60002020202020202020202020202020202076
:101C0000C2AFC2D353D9BF7581C043B20343FF8073
:101C1000752438752503B1C975EF0275E24043F1AB
:101C20008053A47F75D400D2877DFA780379E67C4F
:101C300010752200752300901DD67B0675249875BB
:101C400025013087028142208708D8FBD9F9DCF7CB
:101C500081B4308708D8FBD9F9DCF781B4B189E4C5
:101C600093A3C39A6004DDC381B4DBDBB17B600264
:101C7000812B7B08E493FAA3B15CDBF87A30B15C8A
:101C8000752200752300B17BEAFCEBFDC3ED94FEE9
:101C9000400EB17B8A278B28ED30E0048A828B834B
:101CA000B17B7AC270D8C3ED94FE601350CEBD00F4
:101CB00025EC60097520007521FF0200008100A855
:101CC00027A9280809D804D90281D3B17FEA89AAB3
:101CD000F281C50D81A0C3ED94035049EDA2E092BD
:101CE000007AC5C3E5829400E583941C50902000DF
:101CF00010438F02438F0175B7A575B7F1F030001F
:101D00001FA827A9280809438F01538FFDD804D99C
:101D100002A12089AAE275B7A575B7F1F0A3A10DBC
:101D2000538FFC817C7AC1BD030CE493A3FAB140CC
:101D3000DCF8B138817C817EAA22AB23B15CEBFA5E
:101D4000EA6222752608C3E52313F523E52213F57D
:101D50002250066323A0632201D526EAB1C9B1C986
:101D600075260AEAF4200102D287300102C287B147
:101D7000C9C3134002C201D526EB22B17FEAFB2082
:101D80008702A17F308702A184752608AE24AF2583
:101D9000C3EF13FFEE13FEB1CDB1C9C3EA13308711
:101DA000024480FA30E703632201C3E52313F523DD
:101DB000E52213F52250066323A0632201D526D91C
:101DC000E52265236523F52222AE24AF250E0FDE22
:101DD000FEDFFCD20122424C48656C693437316326
:041DE000F390060175
:00000001FF
